:020000040000FA
:1000000000400110410400003D0D0000410D0000C2
:1000100000000000000000000000000000000000E0
:10002000000000000000000000000000450D00007E
:100030000000000000000000490D0000870F0000D4
:100040004D0D0000510D0000550D0000590D000030
:100050005D0D0000610D0000650D0000690D0000E0
:100060006D0D00005904000059040000000000005C
:100070000000000000000000000000000000000080
:100080000000000059040000590400005904000059
:1000900059040000590400005904000059040000EC
:1000A00059040000590400005904000059040000DC
:1000B00059040000590400005904000059040000CC
:1000C0000448854601F01EFE00480047A7020000D4
:1000D000C046C0460040011010B586B00446BD4879
:1000E000019000216846018201814181C1818181A5
:1000F000FF21013181824182002C08D10821132087
:1001000000F08EFD0921172000F08AFD09E0012C86
:1001100007D10C21062000F083FD0D210E2000F0F8
:100120007FFD01A9204600F09FF906B010BDAA4945
:100130000968491CA84A1160114609680522120382
:1001400091420DD90021A44A1160A44941180978AF
:100150003F2901D13E2100E03F21A04A82181170C1
:10016000704770B505460C46204601F046FD204616
:1001700000F0C6FF01F0D6FB70BD70B505460C4619
:100180002078342829D00CDC142818D004DC01286D
:100190001CD0052823D11AE015280BD018281ED111
:1001A00017E0382814D03D2818D0652812D06628CA
:1001B00015D110E080213C20FFF7D3FF10E0122082
:1001C00001F0D8FA864800F053FE09E008E007E0A5
:1001D00006E005E004E062B602E001E000E000BFF6
:1001E00000BF70BD10B5322001F0C4FA10BDF8B5E3
:1001F00006460C4627786078A1780902401885B237
:10020000122F04D0162F10D0522F1ED112E0042D21
:1002100004D00E2D03D0112D03D101E001E000E048
:1002200000BF00BFFFF7DEFF0FE01C2D00D100BFB5
:1002300000BF0AE01C2D06D1F01E82B2E11C012095
:1002400000F07FFB00BF00BF00BF00BFF8BD00B5DE
:100250008DB0182263A107A801F030FD67A103C982
:100260000691059067A30FCB049301AB07C316213A
:1002700007A801F07BFC05A801F0C4FB0C2101A834
:1002800001F0D0FB0C2101A801F035FCFF20A130CA
:1002900000F03EFFC82001F088FB50216420FFF7EA
:1002A00060FF0DB000BD5B480079012814D15A48A9
:1002B00001F0A4F900F05FFD0120FFF70DFF00F051
:1002C0006DFF01F055F900F017FFFFF7C0FF0121A6
:1002D000132000F01FFC13E0504C601E5049884270
:1002E00000D90CE0601E4F4948610321081F00F04F
:1002F00039F800204B4988610720086100BF00BF22
:1003000000F00DFE2DE04848007D002806D00128B1
:100310001ED002280DD0032822D120E001F079FA66
:1003200000F0C9FD1320FFF702FF402000F0AAFEF5
:1003300016E001F04DFA002806D072B600F021FF59
:1003400003203949087502E000203749087507E0A5
:1003500072B600F01AFF03203349087500E000BFB1
:1003600000BFD0E710B5002819DA304A03071B0F89
:10037000083B9B089B00D2588307DC0EFF23A34059
:100380009A438B071B0E8407E40EA3401A43274BA6
:100390000407240F083CA408A4001A5118E0244ABA
:1003A00003231B02D21883089B00D2588307DC0E5C
:1003B000FF23A3409A438B071B0E8407E40EA34040
:1003C0001A431B4B032424021B198408A4001A514E
:1003D00010BD000034800000340501108080001042
:1003E00054050110020106050312180F18031980A5
:1003F00001080931315858424C450000AC028811BF
:1004000043AC000031313231424C455F5465737466
:1004100000000000004700100005011080A9030043
:10042000FFFFFF0000E000E0204300101CED00E0B3
:1004300000E100E0000000000000000000000000FB
:10044000064800680078002801D0054800470548A4
:100450000047000004470010FEE7000054040000BD
:10046000C1000000A7020000FEB505460C460020B2
:1004700001900026009000270120F749C870084627
:10048000407C80218843F4494874002C04D1F34A0D
:100490002B21F3A001F035F8002D06D0012D04D05A
:1004A000EE4A2C21EEA001F02CF82068002803D0A1
:1004B000F8492068884204D9E84A2D21E8A001F0D3
:1004C00020F8A088002807D0A088042804D0E34A98
:1004D0002E21E3A001F015F8E088002807D0E0887D
:1004E000082804D0DD4A2F21DDA001F00AF8208978
:1004F000002807D02089022804D0D84A3021D8A06B
:1005000000F0FFFF6089402807D06089002804D0F0
:10051000D24A3121D2A000F0F4FFA089002807D0F0
:10052000A089102804D0CD4A3221CDA000F0E9FFE7
:10053000E089002804DDE089FF210131884204DDE3
:10054000C64A3321C6A000F0DCFF208A002804DD63
:10055000208AFF210131884204DDC04A3421C0A035
:1005600000F0CFFF20882901CB4A5052002D12D134
:10057000CA4E290189180E81E0898019290189183C
:100580004881C74E290189184E80208A8019290187
:100590008918888012E0C34E2901BF4A89180E814C
:1005A000E0898019290189184881BF4E29018918DD
:1005B0004E80208A8019290189188880A07A217BA1
:1005C0000843217A0843A17908432179084381210E
:1005D0000843C0B201902901AF4A89180198887375
:1005E000002D04D1B14800909B4F123704E0AF4872
:1005F00011300090984F32370121090700984018B8
:100600000078410849000122120700988018017003
:100610002801A14A115A384600F014FA28019E4ACE
:10062000801801893846083000F00CFA28019A4AEF
:100630008018418938460A3000F004FA2801964AA9
:100640008018018938460C3000F0FCF92801924AE4
:1006500080184188B81C00F0F5F928018E4A8018EE
:100660008188381D00F0EEF928018B4A80184188F6
:10067000B81D00F0E7F9012109070098401800783B
:100680002901854A8918897B0843012212070099AC
:1006900089180870FEBD10B50446002C06D0012C48
:1006A00004D0834A71216EA000F02BFF002C0BD1E7
:1006B00069482030007801210843674920310870DB
:1006C0000846007808700AE063482030407C012129
:1006D00008436149203148740846407C487410BD85
:1006E000F8B504460F4600250026002C06D0012C44
:1006F00004D0704A99215AA000F003FF002C02D1C7
:10070000554D123501E0544D323528460830002849
:1007100004D1684AA02152A000F0F3FE002C09D1B8
:1007200000BF6548807B6449C97B090208430028F3
:10073000F7DC0AE000BF60484030807D5E49403110
:10074000C97D090208430028F5DC28460C3000F07A
:1007500082F9064659483018077028460A3000F0DA
:100760007AF9B04205D12846083000F074F90646FF
:1007700001E0701C86B2314628460C3000F062F968
:10078000F8BDF8B50446002500260027002C06D049
:10079000012C04D04A4AB92131A000F0B2FE002C4D
:1007A00002D12D4D123501E02B4D3235A81D00F040
:1007B00052F906464148301800F04DF90746281D09
:1007C00000F049F9B04204D1A81C00F044F90646F3
:1007D00001E0701C86B23146A81D00F033F938469E
:1007E000F8BD10B50446002C06D0012C04D0354AC3
:1007F000CC211BA000F085FE002C04D12E48123025
:1008000000F029F910BD2C485A3000F024F9F9E71E
:10081000F7B584B004461546002003900026002753
:1008200002900190002C06D0012C04D0264ADC2135
:100830000BA000F066FE0598002804D1224ADD21B5
:1008400007A000F05EFE002C40D10348123001905A
:100850001948123002903DE040800010461D000013
:100860002E2E5C2E2E5C2E2E5C2E2E5C4C6962721F
:1008700061726965725C647269766572735C7561D8
:1008800072745C7963313178785F756172742E634C
:100890000000000010A700006C0501108C0501107D
:1008A0008C0601108C0701108C080110608000007C
:1008B000511D00005E1D00000083001000000110AB
:1008C0006D1D00007F1D0000901D00005848019024
:1008D00058480290029800F0BEF80390002D06D010
:1008E0000398A84202DA002007B0F0BD03950398F0
:1008F000002800D1F8E70198801D00F0ACF806460A
:10090000002714E04C48301801780598C15501982B
:10091000001D00F0A0F8B04205D10198801C00F045
:100920009AF8064601E0701C86B2781C87B20398DC
:100930008742E7DB31460198801D00F083F8384696
:10094000D2E7F7B582B004460026002001900025CA
:10095000002C07D0012C05D0384AFF21033138483C
:1009600000F0CFFD0398002805D1344AFF2104315F
:10097000334800F0C6FD0498002805DC2F4AFF210B
:1009800005312F4800F0BDFD002C02D1284D203D3F
:1009900000E0274D28460830002805D1274AFF21CE
:1009A0000C31274800F0ADFD002C0BD100BF2148D1
:1009B0005A38807B1F495A39C97B090208430028ED
:1009C000F5DC0AE000BF1B481A38807D19491A3946
:1009D000C97D090208430028F5DC28460C3000F0E8
:1009E0003AF80646002718E00398C05D12497118CE
:1009F000087028460A3000F02EF8B04205D128468B
:100A0000083000F028F8064601E0701C86B2019814
:100A1000401C80B20190781C87B204988742E3DBC7
:100A2000314628460C3000F00DF8019805B0F0BDB5
:100A3000728000105A83001000000110A51D0000F4
:100A40006008000070B504460D46257000F059F8A6
:100A50002812607070BD70B504460025002600F0B5
:100A600050F8257800F04DF866783002FF21090231
:100A700008400543284670BD70B50446002500F0C7
:100A800040F8257800F03DF860780002054300F05A
:100A900038F8A07800040543284670BD10B503E07F
:100AA0000B780370491C401C1346541EA2B2002B45
:100AB000F6D110BD0146002201E0521C491C087805
:100AC0000028FAD190B2704700BFFEE710B50021B0
:100AD00006E00F4A00BF1346521E002BFBD1491CF3
:100AE0008142F6DB10BD10B5002107E07D22120126
:100AF00000BF1346521E002BFBD1491C8142F5DB7F
:100B000010BD00BF00BF00BF00BF00BF70470000A6
:100B1000204E000070B504460D4600F005F9202C6B
:100B200000D170BD002D02D0012D12D108E03E2071
:100B3000E106C90E7F4A891852058918087009E034
:100B40003F20E106C90E7B4A8918520589180870B2
:100B500000E000BF00BF00F0E7F800BFE1E770B5BC
:100B600004460D4600F0E0F8202C00D170BD012DA8
:100B700006D0022D0DD0032D14D0042D24D11AE05F
:100B80000020E106C90E6B4A8918520589180870C1
:100B90001BE04020E106C90E664A891882058918C3
:100BA000087012E08020E106C90E624A89184205E9
:100BB0008918087009E0C020E106C90E5D4A89184D
:100BC00052058918087000E000BF00BF00F0ACF8C3
:100BD00000BFCBE730B50146202900D130BDCB06A0
:100BE000980F4A07520F0346AB33012424071B1901
:100BF0001C78012393409C430346AB3301252D070A
:100C00005B191C700346AF332C461B191B7801245B
:100C10009440A3430446AF346419237000BFDDE75A
:100C2000C206D20E434BD2185B05D2181170704722
:100C300070B5024600230024002553075B0FD00641
:100C4000840F0819012636073043057801209840A3
:100C5000284070BD10B50446202C01D1FFF734FFA9
:100C6000E006C00E3449FFF7E3FF10BD70B5024641
:100C70000B46202A00D170BDD406A00F5107490FA2
:100C8000002B02D0012B3AD11CE00446AB340125E5
:100C90002D076419247801258D402C43E5B20446C4
:100CA000AB3401263607A41925700446AF34354607
:100CB0006419257801248C40A5430446AF34A41957
:100CC00025701CE00446AF3401252D0764192478F3
:100CD00001258D402C43E5B20446AF34012636078A
:100CE000A41925700446AB343546641924780125CF
:100CF0008D40AC430546AB35AD192C7000BF00BF2D
:100D000000BFB8E770B504462046FFF7A3FF0546CD
:100D1000002D04D000212046FFF7A8FF03E00121A9
:100D20002046FFF7A3FF70BD00BF00BF00BF00BF9C
:100D300000BF7047808000001C83000000BFFEE7FA
:100D400000BFFEE700BFFEE700BFFEE700BFFEE713
:100D500000BFFEE700BFFEE700BFFEE700BFFEE703
:100D600000BFFEE700BFFEE700BFFEE700BFFEE7F3
:100D700000BF00BF704710B5B648B74908600020F3
:100D800009680861B548B4490968C8600120B249DA
:100D9000096808720020B04909680860B04C601EFC
:100DA000B049884200D90CE0601EAF494861032178
:100DB000081F00F017F90020AB498861072008617F
:100DC00000BF10BD0246002A00D17047A24801684A
:100DD00004E08A4201D10120F7E709690869002887
:100DE000F7D100BFF1E7F0B504460D461646002CDA
:100DF00000D1F0BD2046FFF7E5FF002801D001201B
:100E0000F7E7002B02D19548E06000E0E36072B69E
:100E10006560964800684019206001202072667263
:100E20008D48076804600068076162B60120E0E74A
:100E30000146002900D170478748026809E09142C5
:100E400006D18A4B48681B68C01808600120F2E789
:100E5000126910690028F2D100BFECE700217E4A38
:100E6000106801E0491C00690269002AFAD1704744
:100E700010B50246002A00D110BD7648824201D149
:100E80000020F9E7744801680B460FE08A420BD155
:100E9000002008728B4203D16F4C0869206001E08A
:100EA000086918610120E7E70B460969086900280D
:100EB000ECD100BFE0E710B56D480078002820D0E5
:100EC00000206B4908706448046817E0207A012804
:100ED00013D166492068096888420ED8607A0028D4
:100EE00003D12046FFF7C4FF04E060496068096849
:100EF00040182060E16860698847246920690028FB
:100F0000E4D110BD5449086802E000210172006973
:100F100001690029F9D14F494F4A11607047554A7C
:100F20001278544B5B781B021A43524B9B781B047C
:100F30001A43504BDB781B061A43104600214E4AD9
:100F40001268002A02D14C4A10601AE04A4A12681C
:100F5000824202D9484A10607047474A1268811A93
:100F60000DE0424A1268521C404B1A60424A126815
:100F70002032414B1A60203901223D4B1A70202942
:100F8000EFD200BFE8E700B5FFF7C9FF01203849FD
:100F9000087000BD70B5034600BF334E7569182652
:100FA0005E4334460022304EB1690FE02E4EB069E8
:100FB00088420BD0884202D20E1AB21802E02E1AD2
:100FC0007618B2180146A24200D300E0EEE700BF57
:100FD00070BD10B504467D21C90061430846FFF786
:100FE000D9FF10BD10B5002819DA244A03071B0FDA
:100FF000083B9B089B00D2588307DC0EFF23A340CD
:101000009A438B071B0E8407E40EA3401A431B4B25
:101010000407240F083CA408A4001A5118E0184A39
:1010200003231B02D21883089B00D2588307DC0ECF
:10103000FF23A3409A438B071B0E8407E40EA340B3
:101040001A430F4B032424021B198408A4001A51CD
:1010500010BD00008C09011038050110710D000051
:10106000C05D0000FFFFFF0000E000E03C05011054
:101070004005011000830010440501101CED00E044
:1010800000E100E0434A927B424BDB7B1B021A43A8
:101090000243114600BF3F4B99730A12DA7300BF37
:1010A00070473C4A927B3B4BDB7B1B021A438243DB
:1010B000114600BF374B99730A12DA7300BF7047AD
:1010C0003448807B002801D1012000E00020314914
:1010D000C97B09020843002801D001207047002085
:1010E000FCE700BF00202B498873C87300BF70471E
:1010F00001202949487470470020274948747047E7
:1011000000BF254AC032D0740112117500BF70476C
:1011100000BF204A10770112517700BF704710B509
:1011200000242BE01B484079C006C00EA0421DD011
:1011300018488079C006C00EA04217D01548C07963
:10114000C006C00EA04211D01248007AC006C00EE0
:10115000A0420BD00F48407AC006C00EA04205D076
:101160000C48807AC006C00EA04200D104E0802165
:101170002046FFF755FD00BF601CC4B2202CD1DB18
:1011800010BD10B5FFF7CBFF10BD10B5FFF7C7FFBF
:1011900010BD0000004700102041001000B585B0D0
:1011A000D94800900021684681818180C1804181B9
:1011B0000181FF210131C1810182D44800780028DA
:1011C0000AD1D24988780821FFF72AFDCF4948780B
:1011D0000921FFF725FD0DE0CC480078012809D151
:1011E000CA4988780C21FFF71BFDC84948780D21B2
:1011F000FFF716FDC54908786946FFF735F905B0D0
:1012000000BDC249087070470178C04A11708178EA
:10121000917041785170704770B504460D46AAB27E
:10122000BA4908782146FFF78CFB70BD0FB4F0B5C2
:101230008BB011A8019042E1002400E0641C1098DA
:10124000005D252803D01098005D0028F6D1002C01
:1012500003D021461098FFF7DFFF10980019109077
:10126000109800782528E6D11098401C1090002591
:101270002020039000BF10980178401C109038295E
:1012800030D014DC332928D008DC25296FD0302950
:1012900020D031291FD032296AD11DE034291DD038
:1012A00035291CD036291BD03729F5D119E07029F2
:1012B00073D008DC392916D0582970D0632922D080
:1012C0006429E9D12AE073293CD075295AD07829BC
:1012D000E2D171E000BF00BF00BF00BF00BF00BF90
:1012E00000BF00BF00BF10982038C07F302802D157
:1012F000002D00D103900A20454310982038C07F6C
:1013000030384519B7E7019800680A900198001D28
:10131000019001210AA8FFF77FFFCFE00198006844
:101320000A900198001D019000260A98002805DA0D
:101330000A9840420A900120099001E0002009909B
:101340000A2747E00198006808900198001D019065
:10135000002400E0641C0898005D0028FAD12146B2
:101360000898FFF759FFA5420BD92D1B05E09AE01D
:101370009FE0012166A0FFF74FFF28466D1E002861
:10138000F7D19BE0019800680A900198001D019038
:1013900000260A27002009901CE00EE0FFE70198D4
:1013A00000680A900198001D019000261027002077
:1013B0000990582002900DE000BF019800680A9043
:1013C0000198001D01900026102700200990782028
:1013D000029000BF012403E02046784304466D1EBE
:1013E000204678430A99884207D82146794308461F
:1013F000394600F04DFCA042EED00998002800D0FC
:101400006D1E0998002809D00398302806D12D2296
:101410003046761C04A90A5400200990012D0BD9EE
:10142000102D09D26D1E05E03146761C04AA0398E2
:1014300050546D1E002DF7D10998002804D02D229C
:101440003046761C04A90A5426E0029878280FD169
:1014500021460A9800F01CFC3946009000F018FC68
:101460002C480068425C3046761C04A90A540EE001
:1014700021460A9800F00CFC3946009000F008FC68
:1014800025480068425C3046761C04A90A54394657
:10149000204600F0FDFB0446002CD6D1314604A8BE
:1014A000FFF7BAFE0AE01099481E0121FFF7B4FECB
:1014B00004E0052119A0FFF7AFFE00BF00BF1098A0
:1014C0000078002800D0B7E601900BB0F0BC08BC53
:1014D00004B0184713490870704710B50446114806
:1014E0000078002802D02046FFF7A0FE10BD10B5FE
:1014F00004460C480078012802DD2046FFF796FEDE
:1015000010BD00BFFEE70000348000004805011058
:1015100020000000BC1D0000C01D00004552524FBD
:10152000520000004B05011030B50246E12080005A
:10153000814201DD002030BD002007E00024174B70
:10154000C31801252D072B431C70401CE1239B0071
:101550009842F3DB002007E0145C104BC318012510
:101560002D072B431C70401C8842F5DB0120E2E76D
:1015700010B5EAB0FF22A532094901A800F09EFB90
:10158000FF21A23101A8FFF7CFFF0446002C02D1B2
:1015900004A0FFF74BFE6AB010BD0000FB4700003F
:1015A000C41D00000D0A2A2A2A2A2A2A2A2A2A2A9F
:1015B0002A2A2A70726F66696C6520736572766973
:1015C000636520736574206661696C2A2A2A2A2A59
:1015D0002A2A2A2A2A2A2A2A2A2A2A0D0A00000026
:1015E000A04A1278521C9F4B1A70704710B50446DF
:1015F000282221469C4800F061FB10BD9B490860F1
:10160000704770B505460E469948FFF735FA04460F
:1016100000200CE001210907214309782954611CAD
:101620000C46944A914200D3934C411C88B2B0427C
:10163000F0DB00BF8E490C390C732004000E487398
:101640002002000E887300BF70BD70B50446884844
:101650000C38FFF711FA054685480838FFF70CFAF1
:10166000064600210DE0681C0546834A503A904228
:1016700001D301252D04B54201D1002070BD481CC5
:1016800081B2A142EFDB0120F8E770B504460DE01E
:101690002046FFF7DAFF002801D0012070BD7D252C
:1016A000ED0000BF28466D1E0028FBD1F0E7F8B51D
:1016B00006460D462846FFF7E8FF6D480C38FFF751
:1016C000DBF90446002014E0325C012109072143C4
:1016D0000A70611C0C46684A503A914201D30124B9
:1016E0002404642700BF39467F1E0029FBD1411C1A
:1016F00088B2A842E8DB00BF5D490C390C702004B9
:10170000000E48702002000E887000BFF8BD70B552
:1017100005460E46144659480570002C00D170BD90
:101720005748007D022802D10020554908755348CA
:10173000447022463146801C00F0C0FAA01CC1B2A1
:101740004E48FFF7B4FF00BFE9E710B504466078E4
:10175000002800D110BD4A48007D022802D1002097
:10176000474908756078801CC1B22046FFF79FFF8B
:1017700000BFEFE738B50446424800680090404893
:10178000007D022802D100203D490875684684701A
:101790000321FFF78CFF38BD002070470020704701
:1017A0000020704710B5384C01E000F055F8204695
:1017B000641E0028F9D110BD10B500F04DF810BD21
:1017C00010B500F049F810BD10B500F045F810BD97
:1017D00070B527480838FFF74FF9044624480C38FD
:1017E000FFF74AF90546A54201D1012070BD00204E
:1017F000FCE770B51E48FFF73FF904461C48001F80
:10180000FFF73AF90546AC4201D1012070BD002036
:10181000FCE710B51D4CFFF7ECFF002800D010BD11
:1018200002211A48FFF7EDFE2078002810DD20780D
:101830000D280DDA61781548801CFFF7E2FE60780C
:1018400021788900094B1B685A58A11C904701E078
:1018500000BFFEE700BFE2E700BF00BF00BF00BF60
:1018600000BF704750050110A40901104C0501107C
:101870000C0301100005010050030100940A01103F
:1018800020430010681F000010270000CC09011041
:1018900010B50120FFF76EFF10BD10B50220FFF755
:1018A00069FF10BD0146002007E0F04A121A01232B
:1018B0001B071A4312780A54401C0628F5DB7047B0
:1018C00010B50146002008E00B5CE84A521F821860
:1018D0000124240722431370401C0628F4DB10BDAA
:1018E00030B502461B2901DD002030BD002007E095
:1018F000145CDF4BC31801252D072B431C70401CC3
:101900008842F5DB0120F0E770B505460C46782CDF
:1019100001DD002070BD224629460420FFF7F7FEB6
:101920000120F7E710B50D20FFF724FF10BD10B51B
:101930000E20FFF71FFF10BD10B50F20FFF71AFF95
:1019400010BD10B51020FFF715FF10BD10B52F20EA
:10195000FFF710FF10BD10B51120FFF70BFF10BDF2
:1019600010B5044600BF2078C249C876208800120E
:10197000087700BF00BFA07848776088001288779A
:1019800000BF00BF2079C877A0880012B949203174
:10199000087000BF00BFA0794870E088001288700E
:1019A00000BF1220FFF7E6FE10BDC82806DD00BF0D
:1019B000C821B14A5175002191750EE0172805DD47
:1019C00000BFAD4A50750112917506E000BF1721A6
:1019D000A94A51750021917500BF704710B52120AB
:1019E000FFF7C8FE10BD0146002008E0A04A4C3AAF
:1019F000121A01231B071A4312780A54401C0628A6
:101A0000F4DB704710B50146002008E00B5C984AF3
:101A1000513A82180124240722431370401C0628DF
:101A2000F4DB10BDF3B589B00C4600239348857CE8
:101A300000225CE0924810180126360730430378F4
:101A40008F481018401C30430078089008980928E7
:101A50004BD1E81A0019401C1F2802DD00200BB0F2
:101A6000F0BD00210BE086481018C018401C40183B
:101A700001263607304300786E467054491CA81A78
:101A8000C01A401E8842EEDC00210AE00998465C3C
:101A90007B481018801C401801273F073843067008
:101AA000491CA142F2DB601CC6B275481018012720
:101AB0003F073843067000210BE06846465C7048DB
:101AC0001018C018401C401801273F073843067003
:101AD000491CA81AC01A401E8842EEDCE81A0019F8
:101AE000401C664EB0740120B9E7581C1218AA4277
:101AF000A0DB0020B3E7F3B5FFB0E2B00D46E12173
:101B00008900684600F0F3F85E48C77B5E48C61B54
:101B1000002409E05D48381800190121090708432D
:101B2000007869460855641CB442F3DB5548C57318
:101B3000002408E0E198015D5448201801221207B2
:101B400010430170641CAC42F4DB002409E06846D9
:101B5000015D4E4828180019012212071043017038
:101B6000641CB442F3DB7FB064B0F0BD30B5024614
:101B70000B4600211F2B01DD002030BD00203F4C13
:101B8000607409E010783E4C0C1901252D0764198A
:101B90002070521C481CC1B218465C1EE3B20028DB
:101BA000F0D1364881740120E7E730B502460B4694
:101BB00000211F2B01DD002030BD00202F4C607460
:101BC0000AE010782E4C20340C1901252D076419D9
:101BD0002070521C481CC1B218465C1EE3B200289B
:101BE000EFD12648203081740120E5E721492039D2
:101BF000887370471F494872704700BF1D4A203ADA
:101C000010730112517300BF704770B5B4B0054630
:101C10000E461446002C03DB1748C07DA04202DAB2
:101C2000002034B070BD684605712804010E684676
:101C3000417122463146801D00F040F8A01CC2B21E
:101C400001A90520FFF763FD0120EAE710B5172081
:101C5000FFF790FD10BD10B51820FFF78BFD10BDEC
:101C600010B51920FFF786FD10BD000045410000AA
:101C70005D4500000045001000470010A043001023
:101C8000B3430000004800106F030000104800003C
:101C900030B50B46014600202022012409E00D4604
:101CA000D5409D4205D31D469540491B254695408C
:101CB00040191546521E002DF1DC30BD03460B4382
:101CC0009B0703D009E008C9121F08C0042AFAD2F2
:101CD00003E00B780370401C491C521EF9D2704778
:101CE000D2B201E00270401C491EFBD270470022B4
:101CF000F6E710B513460A4604461946FFF7F0FF0B
:101D0000204610BD064C0125064E05E0E36807CCD1
:101D10002B430C3C98471034B442F7D3FEF7D4F968
:101D2000941F0000B41F000002E008C8121F08C181
:101D3000002AFAD170477047002001E001C1121F4C
:101D4000002AFBD1704755534152545F496E697464
:101D50000055534152545F4465496E6974005553B0
:101D60004152545F53656E64446174610055534140
:101D700052545F52656365697665446174610055CC
:101D8000534152545F4765745278436F756E7400C7
:101D900055534152545F5265616444617461746F7C
:101DA000427566660055534152545F53656E6444F4
:101DB00061746146726F6D4275666600801F000037
:101DC0006C1F00000100020028020018020002033C
:101DD000280102030002002A09756E646566696EB7
:101DE000656404000203280102050002012A0200C2
:101DF0000006000203280102070002042A0810005E
:101E000018001000580208000200280201180900FA
:101E100002032801200A0002052A01000B00020229
:101E20002901000C0002002802F0FF0D0002032827
:101E300001160E0002F4FF14000000000000000074
:101E40000000000000000000000000000F0002027F
:101E50002902000010000203280104110002F5FF0E
:101E6000140000000000000000000000000000005E
:101E70000000000000120002002802E7FE1300022A
:101E800003280120140002C8FE1400000000000016
:101E9000000000000000000000000000000015002D
:101EA0000202290200001600020328010A1700029C
:101EB000C7FE140000000000000000000000000049
:101EC00000000000000000180002032801021900B1
:101ED00002C9FE061122334455661A000200280288
:101EE00017FF1B0002032801041C000202FF14005C
:101EF00000000000000000000000000000000000E2
:101F00000000001D0002032801101E000204FF143F
:101F100000000000000000000000000000000000C1
:101F2000000000001F00020229020000200002033E
:101F300028012021000203FF14000000000000001F
:101F4000000000000000000000000000002200026D
:101F500002290200002300020328010224000205D6
:101F6000FF010000000000000101000030313233A9
:101F70003435363738394142434445460000000085
:101F800030313233343536373839616263646566EF
:101F900000000000B41F0000000501105400000004
:101FA000281D00000820000054050110A4050000B1
:101FB000381D000000000000E11500007B0100005A
:101FC000E1150000E1150000EF010000E11500003F
:101FD000E1150000E1150000E1150000E115000029
:101FE000E1150000E1150000000000000000000005
:101FF000000000000000000000000000010E0600CC
:082000000000000000000000D8
:04000005000000C136
:00000001FF
